:1000000089C300000C94A72EBEC30000BCC300002F
:10001000BAC30000B8C30000B6C30000B4C30000F8
:10002000B2C30000B0C300000C94E52C0C94CD2D9D
:100030000C949A2CA8C30000A6C30000A4C300001F
:10004000A2C30000A0C300009EC300009CC3000028
:100050009AC300000C94C12C96C3000094C3000006
:1000600092C3000090C300008EC300008CC3000048
:100070008AC3000088C3000086C3000084C3000058
:1000800082C3000080C300007EC300007CC3000068
:100090007AC3000078C3000076C3000074C3000078
:1000A00072C3000070C300006EC3000005010902A6
:1000B000A10185020901A1000509190129081500FE
:1000C0002501950875018102050109300931158165
:1000D000257F95027508810609381581257F9501D0
:1000E00075088106050C0A38021581257F95017572
:1000F000088106C0C005010980A101850319012AF4
:10010000B700150126B700950175108100C0050CD8
:100110000901A101850419012AA002150126A002E6
:10012000950175108100C00660FF0961A101096297
:10013000150026FF00952075088102096315002629
:10014000FF00952075089102C005010906A101056F
:100150000719E029E7150025019508750181029529
:1001600001750881010507190029FF150026FF0008
:100170009506750881000508190129051500250156
:10018000950575019102950175039101C009025B06
:1001900000030100A0FA09040000010301010009A5
:1001A0002111010001224400070581030800010913
:1001B00004010002030000000921110100012222B4
:1001C0000007058203200001070503032000010941
:1001D0000402000103000000092111010001227B3B
:1001E000000705840320000112010002000000083E
:1001F00010CB56310003010203011C037600690095
:1002000061006C003A006600360034006300320082
:1002100062003300630000001E034E00790071008D
:1002200075006900730074002000520065007600BC
:100230002E002000330000000E034B006500650017
:10024000620069006F000000040309040000000060
:10025000000000000000000000000000000000009E
:10026000000000000000000000000000000000008E
:100270007E0F00D4FFFFFFC70000007800000000E1
:10028000000000002A2B28000000000000000000F1
:100290000000000000000029000000002C1E342097
:1002A000212224342627252E362D3738271E1F20BD
:1002B0002122232425263333362E37381F04050602
:1002C0000708090A0B0C0D0E0F1011121314151646
:1002D0001718191A1B1C1D2F3130232D3504050644
:1002E0000708090A0B0C0D0E0F1011121314151626
:1002F0001718191A1B1C1D2F3130354C35001E00E4
:100300001F002000210022002B0014001A0008000A
:1003100015001700290004001600070009000A0054
:10032000E1001D001B000600190005002552E00039
:10033000E200E30023522C002300240025002600C5
:1003400027002A001C0018000C00120013004C00AB
:100350000B000D000E000F003300340011001000E0
:1003600036003700380028002C002452500051007D
:1003700052004F0035001E001F0020002100220007
:100380002B0014001A00090013000A0029000400C1
:100390001500160017000700E1001D001B000600F5
:1003A000190005002552E000E200E30023522C0072
:1003B000230024002500260027002A000D000F003E
:1003C00018001C0033004C000B00110008000C004A
:1003D000120034000E0010003600370038002800EC
:1003E0002C0024525000510052004F0035001E00D6
:1003F0001F002000210022002B00340036003700AF
:1004000013001C00290004001200080018000C0052
:10041000E100330014000D000E001B002552E00027
:10042000E200E30023522C002300240025002600D4
:1004300027002A0009000A00060015000F004C00E2
:1004400007000B001700110016003800050010000F
:100450001A0019001D0028002C00245250005100E1
:1004600052004F0035021E021F022002210222020A
:1004700035021E021F022002210222024C003A0015
:100480003B003C003D003E0005784000410042003A
:1004900043004400010001000100010001000100CF
:1004A000230224022502260227022A002302240214
:1004B0002502260227024C003F002D022E022F02A9
:1004C000300231024500320264024A004D00010050
:1004D00001000100AB00AA00A900AE0035001E001B
:1004E0001F0020002100220035001E001F002000F8
:1004F000210022004C003A003B003C003D003E0041
:10050000010040004100420043004400010001009E
:100510000100010001000100230024002500260045
:1005200027002A00230024002500260027004C0075
:100530003F002D002E002F0030003100450032001A
:1005400064004B004E00010001000100AB00AA0056
:10055000A900AE003A003B003C003D003E003F00D9
:100560000100007C4278437846784578010001001C
:100570000100807481741570010001000100010008
:100580000100010001000100010001000100010063
:10059000400041004200430044004500487847784D
:1005A0004A78497801004C0014704052415242523E
:1005B0000100010001000100010001000100010033
:1005C000010001000100010001000100FD377A581F
:1005D0005A000004E6D6B4460200210116000000CD
:1005E000742FE5A3E003B201085D003D888986D33E
:1005F000DC0AE842C3249258425AFA4B42162C5F56
:10060000542BA3199BCDF09E3ED52B7388208A27AF
:1006100002C28C6C91863337C68276CB812B45B073
:100620004557660343EA9B6B19E8B1AAA5E31F2C63
:1006300065784B4034F572DD554C0E88976FFB9210
:100640000FB4A5F05BB19A2B1D54928E8272F648BE
:10065000E7B4799F489284ADB1C6FC79939A8D1C1A
:1006600035FF1B43F6C6C36EBA331667230739003E
:1006700080DCF0C90C81E00A7D63DD01534C5B95A1
:10068000B69BDD20F18041788D582E31A49DE6E4A3
:1006900022C3AEFD3C42DB72E04C0613E4B985296F
:1006A000FF5AE82552FB2F1DAE76F50CE6A9333E26
:1006B000C260D50808F250A7490CB73F7F5CCCBB9D
:1006C0008B1564DEBF6F0059C9DDAAEC69D00951F2
:1006D000F1D362269E135492CC3819E51A9CEAD3C2
:1006E00022865F6703DF3AED5FB76A10E5AD968D4E
:1006F0004D7F0000B6C38E336581AEE60001A402D3
:10070000B3070000B4239031B1C467FB02000000BE
:100710000004595A11241FBECFEFDAE0DEBFCDBF6F
:1007200004B603FE19C08091F2039091F303A091E7
:10073000F403B091F5038730904BA740B04B61F4C0
:100740001092F2031092F3031092F4031092F50347
:10075000E0E0F8E3099500C011E0A0E0B1E0E6ECCC
:10076000F2E602C005900D92A43CB107D9F723E050
:10077000A4ECB1E001C01D92A23FB207E1F70E94D4
:10078000A1250C94EE303CCC9C0191509F31B0F4EB
:10079000832F817034FF0AC08295807F31FD806293
:1007A00032FD806433FF0BC08068089531FD8260A4
:1007B00032FD846033FF03C08860089580E00895AF
:1007C000CF93DF93EB01E0DFFE010995DF91CF913D
:1007D0000895982F92959F7061F420E0982F892FAB
:1007E0008695869511F02E5F982F892F8695820F1A
:1007F000089524E0F4CF8093A70308958093A8037D
:10080000089521E001C0220F8A95EAF78091A8039C
:10081000822BF4CF21E001C0220F8A95EAF7822FC4
:1008200080959091A8038923E9CF292F9A3090F5DC
:10083000863080F590E036E0239F800D911D1124D5
:1008400051E081FD54E080FD550F82FD529523E07B
:10085000969587952A95E1F7FC01EE0FFF1FE80FAB
:10086000F91FE859FD4F20E030E070E04191DF01D1
:10087000CB01022E02C0969587950A94E2F78695E1
:10088000880B8427852384278E932F5F3F4F233047
:10089000310561F70895292F9A3070F5863060F59B
:1008A00090E036E0239F800D911D1124682F677022
:1008B00023E0969587952A95E1F7FC01EE0FFF1F3F
:1008C000E80FF91FE859FD4F40E050E080E021912A
:1008D00030E0062E02C0369527950A94E2F7217083
:1008E000042E01C0220F0A94EAF7822B4F5F5F4F5C
:1008F0004330510561F7089580E008959091A80371
:1009000021E030E0F90101C0EE0F8A95EAF7D90144
:1009100001C0AA0F6A95EAF7EA2B01C0220F4A9597
:10092000EAF7892F8E23E81303C0892F822B66CF25
:100930002095822F8923FBCFE091B0039091AF03E4
:10094000E91302C080E008959F0157E0E59FF001A0
:100950001124EF54FC4F5181561306C05081581397
:1009600003C05581541305C02F5F3F4FF901E77055
:10097000E7CF81E008958091B0032091AF03281361
:1009800001C0089501968770FACF9091AA038095CF
:1009900089238093AA03282F277081F4891771F087
:1009A0009091F10392FF0AC086958695869532DF75
:1009B0001092AA031092AB031092AC030895909189
:1009C000A503982B9093A50308958095982F809167
:1009D000A50389238093A50308958091A40381151D
:1009E00031F01092A4031092AD031092AE0308955B
:1009F000803E9105D1F1C8F48133910509F481C09D
:100A000048F48932910509F471C08A32910509F4DC
:100A10007FC0089589339105E1F082389105C9F0CE
:100A20008533910509F45DC00895843E9105D1F1A7
:100A300048F4823E910531F1833E910541F181EE0A
:100A400090E00895863E9105C1F1873E9105F1F150
:100A500008952091F003237009F064C02091F10300
:100A600023FF14C089E290E008952091F00320FD57
:100A700045C03091F10330FF09C024FD24C083EE4E
:100A800090E008952091F00322FDF7CF0895209182
:100A9000F00322FD44C03091F10330FD43C024FF38
:100AA000F5CF11C02091F10321FFF0CF8091F00329
:100AB00084FD09C087EE90E008952091F00323FFA4
:100AC000E5CF24FFF7CF80E090E008952091F00378
:100AD00023FD2BC03091F10331FFE1CF84EE90E094
:100AE00008952091F00325FFD1CFBCCF2091F003D2
:100AF00025FD1EC02091F10323FFC8CF89E390E0BC
:100B000008952091F00326FFC1CF8AE290E0089576
:100B10002091F00326FFBACF81E390E0089582EEA2
:100B200090E0089580EE90E0089586EE90E00895BC
:100B300085E390E008959091F00392FF10C041E0AA
:100B4000282F2471243009F040E031E0282F28714B
:100B5000283009F030E0431711F02CE0822793FF92
:100B600010C041E0282F2471243109F040E031E029
:100B7000282F2871283109F030E0431711F02CE0BC
:100B800082273091F10330FF10C051E0282F2171EE
:100B9000213009F050E041E0282F2871283009F079
:100BA00040E0541711F029E0822731FF10C041E0E6
:100BB000282F2171213109F040E031E0282F2871E0
:100BC000283109F030E0431711F029E0822794FD25
:100BD000877E08950F931F93CF93DF9309DFEC0176
:100BE000D23508F04DC0D03508F0C3C0C03ED105A5
:100BF00030F5CD3CD10508F09AC0C83AD10578F45B
:100C0000C53AD10508F090C0C130D10599F1CE01A7
:100C10000497813A910570F1C0E0D0E02BC0CE017D
:100C2000885A91094B97C0F7C85AD0E0CC0FDD1F06
:100C3000C95ADE4F0990D881C02DD4641BC0D0346E
:100C400090F4D03208F0A8C0C83ED10598F0CE018B
:100C500091509F3108F78D2F6EDF082F8C2F90E079
:100C6000C7DE902B54C08C2F90E0C2DEDF70C82FFF
:100C7000D92BD06ACE01DF91CF911F910F910895AA
:100C8000C03882E5D807B8F5C03682E5D80708F045
:100C900056C0C03482E5D807C8F4C03282E5D80710
:100CA00008F047C08C2F8695869520E2829FC00170
:100CB0001124C37021E030E002C0220F331FCA9517
:100CC000E2F7E901C82BD92BDD68D4CF8C2F8695AC
:100CD0008695877020E2829FC0011124C37021E0B5
:100CE00030E002C0220F331FCA95E2F7E901C82B9A
:100CF000D92BDC68BFCFC03C82E5D80750F48C2FDD
:100D00008F71C03AD24580F5982F84EF906AEC013C
:100D1000B1CFCE01805C9245809708F07DCFDC2F6B
:100D2000DF71C0EFD06AA6CFA497D064A3CFD065FF
:100D3000A1CF8C2F8F71D82FC1EFD06A9BCF8C2F72
:100D400086958695877020E2829FC0011124C3702A
:100D500021E030E002C0220F331FCA95E2F7E9011B
:100D6000C82BD92BDA6886CFE6DEC0E0D82FD06258
:100D700081CF8C2F8F71DFDE93E0CC0FDD1F9A9532
:100D8000E1F7DF70282F84FF04C090E1899F900174
:100D90001124C22FD0696ECF8D2F8F71CCDE082F1A
:100DA0008C2F90E025DE902BEC01E1CF80E00895C0
:100DB000F894E82FE295EF70F0E041A18F7021E008
:100DC00001C0220F8A95EAF7922F9095942391A360
:100DD00092A1822F892B82A3789408950F931F9359
:100DE000CF93DF93883080F581112FC090918000E0
:100DF0009F77909380002091860030918700A82FE4
:100E0000B0E00E94E92F27E030E040E050E00E948F
:100E10002E30E901FA0180918600909187006CE004
:100E200070E00E9407306217730798F0C90169E00B
:100E300070E00E9407307093890060938800DF9112
:100E4000CF911F910F91089587E090918000906855
:100E5000D0CF8091860090918700209186003091BC
:100E600087008901209186003091870066E070E05C
:100E70000E940730C60FD71FE11DF11D85E0CC0F82
:100E8000DD1FEE1FFF1F8A95D1F7C80166E070E0F5
:100E90000E94073040E050E0260F371F411D511DD2
:100EA000BE01CF010E942E30E901FA018091860037
:100EB000909187008C01B901CA010E94F82F9B0113
:100EC000AC01D8010E945D309B01AC01BE01CF0195
:100ED0000E94F82F770FBB27AA27881F991FAA1FE8
:100EE0002091860030918700281739071A061B06C3
:100EF00020F48091860090918700BC019CCF8830BF
:100F000008F087E0209193022770982F990F990F8E
:100F1000990F922B9093930221E0983008F420E0EF
:100F20009091930220FB90F99093930257CFE09118
:100F30005E02F0915F02309739F00284F385E02D74
:100F4000309711F060E20995089581152CE792071A
:100F500041F42091120230911302232B11F480E00E
:100F600090E00895EDE1F3E080E090E06EE574E25A
:100F700041E854E224EF34E2668377834087518767
:100F800022873387868797870196709688309105E8
:100F900099F70895FC01AC014B5F5F4F8FEF61E360
:100FA0009191892728E030E0982F990F87FF09C099
:100FB000892F862721503040B9F7E417F50781F7CC
:100FC0000895892FF7CFFC018481862351F4928103
:100FD0009115B9F06923808583FF05C081E0611117
:100FE0000FC080E00895292F22952F709F70292B24
:100FF000962F92959F706F70962B81E02913F1CFF9
:10100000089581E008950F931F93CF9301E0082E78
:1010100001C0000F0A94EAF7C091A3039C2F90230C
:10102000A9F49091AA03969596959695891306C072
:101030001092AA031092AB031092AC03E2DBC0271C
:10104000C093A303CF911F910F910895E3DBF7CFD6
:10105000382F25EB3203C001112497FF04C08058BC
:101060009109892F089580589F4FFBCF809182026C
:1010700080FD14C081FD14C082FD16C080918102E4
:10108000811581F08E3180F420E5829FC00111240A
:101090006EE170E00E941B30862F089584E1089570
:1010A00088E2089588E0089580E50895809182029D
:1010B00080FD17C081FD17C082FD19C0809180029C
:1010C000811599F0883298F428E0829FC00111249C
:1010D00068E270E00E941B306115710551F0862FA7
:1010E000089562E0FCCF64E0FACF61E0F8CF68E0F9
:1010F000F6CF81E008954115510511F0FA010995E7
:10110000089580915202811571F0E0915E02F09194
:101110005F02309739F00190F081E02D309711F0A7
:101120000995089580E00895A3E0B0E0EAE9F8E0C9
:101130000C94C22F2091E7013091E801281739075C
:10114000B1F08093E7019093E801E0915E02F091A5
:101150005F02309761F00084F185E02D309739F01F
:1011600023E029838A839B83CE01019609952396E8
:10117000E2E00C94DE2FA3E0B0E0E1ECF8E00C94A8
:10118000C22F2091E5013091E60128173907B1F00F
:101190008093E5019093E601E0915E02F0915F0299
:1011A000309761F00084F185E02D309739F024E02C
:1011B00029838A839B83CE01019609952396E2E0D9
:1011C0000C94DE2FA8ECB1E0EFEF90E02C918217A9
:1011D00059F01196EF3F19F4211101C0E92F9F5FDB
:1011E0009630A1F7EF3F09F40895FE2FFF0FFF0B94
:1011F000EA53FE4F82830895E8ECF1E09191891360
:1012000002C0DF011E9291E0EE3CF907B9F70895A4
:101210008091010108952FB7F8948091E101909198
:10122000E201A091E301B091E4012FBF08959091F4
:10123000F10392FF0EC0982F990F990F990F962BDB
:101240009093AA03DEDAE7DF8093AB039093AC03BD
:101250000895D7CA9091A403292F282359F0809587
:1012600089238093A40390E08111D5DF8093AD039F
:101270009093AE030895CFDF9C01909185028091F9
:101280008602982B21F020930B0230930C02909150
:10129000870280918802982B21F0209309023093D5
:1012A0000A02E0915E02F0915F02309759F00680E9
:1012B000F781E02D309731F082E08093830283E85C
:1012C00092E009950895611509F440C0E82FED5C9E
:1012D000E33148F4F0E0E051FF4C0C945030C6DEAE
:1012E000819580938602C7CFC1DEFBCFBFDE81959B
:1012F00080938502F8CFBADEFBCFD8DE80938702D9
:10130000F2CFD4DE8195FACFD1DE81958093880229
:10131000EACFCCDEFBCF815D990B21E001C0220F2B
:101320008A95EAF780918402822B80938402DBCF36
:1013300080918202816080938202D5CF8091820267
:101340008260F9CF809182028460F5CF409185025E
:101350008D3C59F48091860287FF0DC01092860261
:10136000411559F41092810208C08E3C81F480919D
:10137000860218169CF3411581F0809187029091A6
:101380008802892B09F0AFCF10928002ACCF8F3C3E
:1013900041F447FFF0CF10928502809186028115BB
:1013A000E0CF803D19F41416B4F3E5CF9091870295
:1013B000893D29F41916FCF610928702DCCF8A3D8C
:1013C00019F497FFD8CFF8CF909188028B3D29F47C
:1013D00097FFD1CF10928802CECF8C3D19F4191609
:1013E000CCF3C9CF982F915D983078F4815D990B3B
:1013F00021E001C0220F8A95EAF7822F8095909113
:101400008402892380938402B6CF8D3D31F480918C
:1014100082028E7F80938202AECF8E3D21F4809136
:1014200082028D7FF7CF8F3D09F0A5CF8091820298
:101430008B7FF0CF2FB7F8946091E1017091E201BA
:101440008091E3019091E4012FBF089580915202B1
:10145000811539F0EFDF462F572FBC01CB01BA01C0
:101460000895E8DFDC01CB01409154025091550210
:101470006091560270915702480F591F6A1F7B1FD7
:10148000EDCFCF92DF92EF92FF92CF93DF93EC01FB
:10149000C0901703D0901803E0901903F0901A033E
:1014A000C9DFDC01CB018C199D09AE09BF09843F5E
:1014B0009140A105B10508F1BDDF6B017C0182E31C
:1014C00090E0C0920502D0920602E0920702F092EC
:1014D000080280930102909302021092030210927C
:1014E0000402CE01C093150390931603DF91CF91B0
:1014F000FF90EF90DF90CF90089584EF91E0E1CFDF
:101500000895FC012091D7013091D80126173707A3
:1015100048F06115710529F49091E8009E77909349
:10152000E8009B0190E02115310541F4911106C0BE
:101530008091E80082FF32C080E00895809114021B
:101540008115C1F18530C1F18091E80083FD30C083
:101550008091E80082FDECCF8091E80080FFE3CF2E
:101560008091F3004091F200582F2115310519F0B8
:101570004830510558F091E04830510509F090E0AD
:101580004091E8004E774093E800CDCF8191809361
:10159000F100215031094F5F5F4FE7CF8091140276
:1015A000811541F0853041F08091E80083FFC0CF84
:1015B00081E0089582E0089583E00895982F909344
:1015C000E900891771F07091EC002091ED005091C5
:1015D000F00021FD09C09F5F973089F78093E900F3
:1015E0000895762F242F50E03091EB003E7F30930A
:1015F000EB003091ED003D7F3093ED003091EB003A
:1016000031603093EB007093EC002093ED00509329
:10161000F0002091EE0027FDDECF08958091D101EA
:1016200087FF13C08091E80082FF06C08091E80028
:101630008B778093E8000895809114028111F2CF96
:101640000895809114028115D9F38091E80080FFFC
:10165000F8CF8091E8008E77ECCF2091E4003091B4
:10166000E50095E6A9012091EC00822F817020FF12
:1016700006C08091E80080FF06C080E008952091B8
:10168000E80022FD1AC080911402811589F085308E
:1016900089F08091EB0085FD0FC02091E40030912E
:1016A000E50042175307F9F29150E1F684E00895FE
:1016B00082E0089583E0089581E00895CF93DF9359
:1016C000C8EDD0E088818F7E8883E7EDF0E08081EF
:1016D0008160808384E082BF81E08093D001888133
:1016E0008E7F8883E2EE10821092DA00A1EEB0E0E5
:1016F0001C9288818F77888388818068888388811D
:101700008F7D888319BC109214021092CF01109221
:10171000F5011092CE01A0EE8C918B7F8C93888185
:101720008160888342E060E080E048DFA1EEB0E0C5
:101730008C918E7F8C93E2EEF0E0808181608083DB
:10174000808188608083E0EE80818E7F80838881C5
:1017500080618883DF91CF910895E8EDF0E080818A
:101760008E7F80831092E2001092DA001092E100E6
:10177000A0EEB0E08C9181608C9380818F77808324
:1017800019BCA7ED8C918E7F8C9380818F7E808396
:101790001092D0010895A0E0B0E0E1EDFBE00C94E0
:1017A000BA2F7C016B015A01809135020AE010E0EA
:1017B0008A3010F001E010E0C1E0D0E0B601C701CE
:1017C000F5010995811115C021960C171D078CF0A4
:1017D000CC9F9001CD9F300D300D112480E090E022
:1017E00045E34A95F1F70000019682179307C1F788
:1017F000E5CFCDB7DEB7EAE00C94D62F81E0809339
:10180000E00080E28093D8001092C9008FE19EE44E
:101810000197F1F700C00000A7E0B0EBCD01809385
:10182000F2039093F303A093F403B093F50388E1DC
:101830009CE00FB6F894A895809360000FBE90933B
:101840006000FFCF0F931F93CF93DF93EB018A01CB
:1018500090911402943059F58093E9008FEF9091A4
:10186000E80095FD06C095ED9A95F1F700008150CE
:10187000B1F78091E80085FF1AC0EFDE811112C038
:101880008091E80085FD06C08091E8008E77809306
:10189000E800F3CF88818093F1000150104011F0EF
:1018A0002196EECF8091E8008E778093E800DF915B
:1018B000CF911F910F910895603229F440E250E0DA
:1018C000BC0182E0BFCF0895CF93DF93EC0148E0E5
:1018D00050E0BC0181E0B6DF88E0FE01A9EDB1E097
:1018E00001900D928A95E1F7DF91CF91089546E03E
:1018F00050E0BC0184E0A6CF43E050E0BC0184E0AE
:10190000A1CFCF93DF93C1E001C0CC0F8A95EAF756
:101910006C2F83E090E00E94B9308C2F0E94FB0373
:10192000DF91CF910895FC01608186E090E00C94F6
:10193000B9308091930280FD11C081608093930241
:10194000813019F489E08093930283E992E0EBDF20
:101950008091930286958695869540CA08951F9337
:10196000CF93DF93122F8630E0F46A30D0F4463004
:10197000C0F4C42FD0E0CC0FDD1F2CE0629FC00D5F
:10198000D11D112498E7899FC00DD11D1124632F0B
:10199000CE0189960E94B930612FCE018A960E94AD
:1019A000B930DF91CF911F9108959091F10392FB8F
:1019B000222720F9281779F080FB92F99093F10300
:1019C0006091F0037091F10384E090E00E94D330C5
:1019D00082E00C94C5040895CF93C091A503809133
:1019E000A903C82B8091A4038115F1F014DC209188
:1019F000AD033091AE03821B930B8838934110F0F6
:101A00000E94ED048091A403C82B20E088EC91E0B3
:101A1000FC013081019631112F5F31E08E3C93073C
:101A2000B9F721110E94ED048091990280958C23D1
:101A300090919802892B8093C60148E050E060E6BF
:101A400072E086EC91E00E947030892BB9F088E05A
:101A5000E6ECF1E0A0E6B2E001900D928A95E1F7A4
:101A6000E0915E02F0915F02309741F00280F381D5
:101A7000E02D309719F086EC91E00995CF9108950B
:101A80001092A503E8ECF1E086E011928A95E9F75F
:101A900080E090E049DB80E090E06DDB1092A903EC
:101AA0009BDFE3E8F2E086E011928A95E9F7109275
:101AB00081021092800210928202DDCBE1DF8FEF73
:101AC00094E32CE0815090402040E1F700C00000FA
:101AD00088E19CE00FB6F894A895809360000FBE53
:101AE00090936000FFCFAAE2B0E0E9E7FDE00C943C
:101AF000C12F81ED91E0FC0101962091F10020833E
:101B000021E0893D9207B9F78091D201893009F42B
:101B100057C0C8F4823009F4B3C0833009F483C0DD
:101B2000813081F18091E80083FFE7C08091D1018D
:101B30009091D2019A3008F0E0C0E92FF0E0ED5F1B
:101B4000FE4C0C9450308A3009F48AC08B3051F727
:101B50008091D101813231F78091D5019091D601E8
:101B6000892B01F78091E800877F8093E80056DD9C
:101B700081E09091D301911101C080E08093020136
:101B80007FDFD0CF8091D101813A61F68091E8006A
:101B9000877F8093E8008091D5019091D601892BB1
:101BA00059F060E080E090E070E0ABDC8091E8000C
:101BB0008B778093E800B6CF68E089ED91E0F4CFB1
:101BC0008091D101813209F0ADCF8091D501909102
:101BD000D6018D7F892B09F0A5CF8091E800877F02
:101BE0008093E8008091E80082FF18C02091F30004
:101BF0008091F200922F029731F48091F1008130B0
:101C000011F0863021F48091F100809301018091E0
:101C1000E8008B778093E80001DD84CF8091140287
:101C20008111E0CF7FCF8091D101813A09F07ACF45
:101C30008091D5019091D601892B09F073CF8091C5
:101C4000E800877F8093E8008091E80080FFFCCF68
:101C5000809102018093F1008091E8008E77DACFC5
:101C60008091D101813209F05DCF8091E800877FBA
:101C70008093E800D3DC8091D4018093000152CF9F
:101C80008091D101813A09F04DCF8091E800877FA2
:101C90008093E8008091E80080FFFCCF80910001F4
:101CA000D9CF803889F0823841F58091D5018F7085
:101CB000873018F58093E9008091EB0085FB882739
:101CC00080F91092E90006C08091F501880F90918B
:101CD000CE01892B9091E800977F9093E800809344
:101CE000F1001092F1008091E8008E7723C08111FD
:101CF00016C08091D301813009F18091E80083FF03
:101D00000AC08091E800877F8093E8008091EB0013
:101D100080628093EB00AA96E3E00C94DD2F823082
:101D200061F78091D301811579F01092E9008091DB
:101D3000E800877F8093E80071DCDFCF933009F003
:101D400080E08093F501F1CF8091D5018F70282F2D
:101D50002150263090F68093E9002091EB0020FF7F
:101D6000E4CF933031F48091EB0080628093EB00FC
:101D7000DCCF9091EB0090619093EB0021E001C0EB
:101D8000220F8A95EAF72093EA001092EA008091E8
:101D9000EB008860EBCF8111B0CF8091D3018F77BA
:101DA000182F8091E3008078812B8093E30080914D
:101DB000E800877F8093E80031DC8091E80080FFB5
:101DC000FCCF8091E30080688093E30083E01111F1
:101DD00001C082E08093140290CF8058823008F0D6
:101DE0008CCF8091D3019091D4018C3D23E0920758
:101DF00089F583E08A838AE289834FB7F894DE010C
:101E0000139620E03EE051E2E32FF0E050935700BC
:101E1000849120FF03C082958F703F5F8F708A305E
:101E2000B8F0895C8D931D922F5F243169F74FBF05
:101E30008091E800877F8093E8006AE270E0CE013D
:101E400001965FDB8091E8008B778093E80055CFA7
:101E5000805DE8CF292F30E02330310509F44EC0F2
:101E600078F52130310509F486C08BE590E0EDE886
:101E7000F1E02230310509F040CF2091E800277FC2
:101E80002093E8002091D7013091D8018217930761
:101E900008F49C0140E02115310509F071C04111A1
:101EA0006FC08091E80082FDCDCF80911402811532
:101EB00049F2853039F28091E80083FFF2CFC2CF3A
:101EC0008091D5019091D6012132310509F444C0A9
:101ED0002232310509F011CF8330910508F00DCF82
:101EE000FC01EE0FFF1FE25CFE4F0190F081E02D40
:101EF000855C9E4FDC018C9190E010C0282F30E073
:101F0000823011F12330310568F4232BA9F4E8E481
:101F1000F2E0E4918E2F90E0E8E4F2E0009709F41B
:101F2000ECCEABCF09F0E9CEEAEFF1E0E4918E2FF1
:101F300090E0EAEFF1E0F2CFE8E3F2E0E4918E2FF7
:101F400090E0E8E3F2E0EACFE8E1F2E0E4918E2FFE
:101F500090E0E8E1F2E0E2CF8330910508F0CDCEE9
:101F6000880F991FFC01EC5BFE4F0190F081E02D82
:101F700089E090E082CF82E190E0E8EEF1E07DCF71
:101F800080911402811509F45DCF853009F45ACF90
:101F90008091E80083FD56CF8091E80082FD81CFDB
:101FA0008091E80080FF77CF4091F3008091F200AC
:101FB000942F2115310519F08830910550F041E03A
:101FC000089709F040E08091E8008E778093E80060
:101FD00062CF44914093F10031962150310901962E
:101FE000E8CF803809F089CE8091E800877F809320
:101FF000E8008091CF018093F10075CE81117DCEF4
:102000008091D301182F823008F077CE8091E800BC
:10201000877F8093E8001093CF0100DB1115D9F082
:1020200084E08093140242E061EC81E0C7DA42E28E
:1020300061EC84E0C3DA42E261EC82E0BFDA42E2C2
:1020400060EC83E0BBDA80911402843051F482E0CA
:102050008093030152CE8091E30087FDE1CF81E0C0
:10206000E0CF81E0F5CFCF93C82F8115A1F0823862
:10207000A1F447D881FD0FC089E3A4D8ADDC8FEF70
:1020800097EE23E0815090402040E1F700C000002F
:1020900089E3B2D8A1DCCF910895833889F431D88F
:1020A00080FDF9CF83E58ED897DC8FEF91EE24E0A9
:1020B000815090402040E1F700C0000083E5E9CF67
:1020C000843889F41ED882FDE6CF87E47BD884DC8F
:1020D0008FEF91EE24E0815090402040E1F700C066
:1020E000000087E4D6CF8450813A70F4E8ECF1E048
:1020F0008EEC91E02081C217A9F131968E179F07CF
:10210000C9F78C2F5FD8C6CF8C2F805E883050F4F3
:1021100081E0C1FD84E0C0FD880FC2FD82950E9470
:10212000DF04B8CF8C2F855A833030F48C2F845243
:10213000990B0E949408AFCFEC2FE85AEB3148F48A
:10214000F0E0EE0FFF1FE357FE4F8081918113D81F
:10215000A2CF8C2F8D5C833108F09DCF61E08C2F56
:10216000B2D899CF8C2F48D837DCCBCFCF93DF9321
:10217000EC01805E9109089720F06DE371E12097F2
:1021800011F461E371E1CE010E94E0038C2F6BDF5B
:10219000DF91CF910895811509F44CC0823851F434
:1021A0000E94810881FF46C089E30CD815DC89E3D1
:1021B00023D812CC833849F40E94810880FF3AC0AA
:1021C00083E500D809DC83E5F3CF843851F40E941D
:1021D000810882FF2FC087E40E94E208FDDB87E4CC
:1021E000E7CF982F9450913A18F3982F905E98303B
:1021F00058F4982F81E091FD84E090FD880F92FDC6
:1022000082950E94E504D5CF982F955A933020F4FB
:1022100080E090E00C949408982F985A9B3120F419
:1022200080E090E00C94BB08982F9D5C933110F4F3
:1022300060E049C808951F93CF93DF93182FEB01F7
:1022400012DF209731F4812FA6DFDF91CF911F910C
:1022500008958FE99FE00197F1F700C000002197F2
:10226000F0CF811519F00E94DF04B6CB08958115D7
:1022700019F00E94E504B0CB0895811531F09091DA
:10228000A903982B9093A903A7CB0895811539F042
:1022900080959091A90389238093A9039DCB0895EC
:1022A00080919402811521F082E2F0DF1092940275
:1022B00008951F93CF93DF93182FA0911303B0912C
:1022C0001403109709F446C01092150310921603D8
:1022D00010929902109298021696CD91DD9118975E
:1022E0009E0131503F3100F4D1E0C11101C0D0E076
:1022F0001996ED91FD911B97309731F01B966D91DA
:102300007D9180E00995D823D11539F08C2F845028
:10231000813A20F58C2F0E94FC081115A1F0E09164
:102320001303F0911403808584FD0DC08091120386
:10233000811549F0808191819C01215031092F3311
:102340003E4708F49ED848DB109213031092140302
:1023500010921203DF91CF911F9108953DDB8C2FD6
:102360001ADFDBCFCF93DF93EC014A855B856E8567
:102370007F850E947B089B8190958091A90389238A
:102380008093A9038C810E94E50426DB86E01992E4
:102390008A95E9F7DF91CF910895CF93DF93EC0110
:1023A0008D8181FD13C082608D838091A9039B8103
:1023B000892B8093A9038C810E94DF040DDB488563
:1023C00059856E857F85CE010E947B0810929D0302
:1023D00010929E038D8180FD02C0CE01C3DFDF918C
:1023E000CF910895AFE0B0E0E8EFF1E10C94B92FA0
:1023F000FE013196DF018AE01D928A95E9F78CE4AF
:10240000C82E81E0D82E7F01AE2E9F2C07E511E06B
:10241000F60181916F018F3F09F43DC0F894E82FD8
:10242000E295EF70F0E021A18F7041E001C0440F10
:102430008A95EAF7922F942B91A392A1842F8095ED
:10244000892382A3789400C0E1E5F1E031E0B12C6A
:1024500021912F3F79F0A22FA295AF70A05EB0E03E
:102460008C9190E02F7002C0959587952A95E2F7A0
:1024700080FF7FC080E0B82A330F0E171F0741F797
:10248000F60182918F3F11F00E94D80680EA8A956A
:10249000F1F7F701B0828FEFE81AF80A81E591E0D1
:1024A0008C159D0509F0B4CF4AE050E06A2D792DD6
:1024B00088E492E00E947030009749F02AE0EA2D0B
:1024C000F92DA8E4B2E001900D922A95E1F7009170
:1024D000470210E0035C1D4F892B09F44CC081E0DA
:1024E00080933C020E940B0980933A0290933B0236
:1024F00080915202811509F498C07E018BE0E80EAC
:10250000F11CF70185E011928A95E9F78091350277
:102510008A3008F054C047E454E1B701C8013BD900
:10252000811509F470C04AEE53E1B701C80133D9EF
:10253000811509F468C041EE54E1B701C8012BD9F7
:10254000811509F460C0109235028091390290E043
:1025500045E050E0B701835C9D4F0E94703021E060
:1025600020933802892B09F041C02F96EBE00C94A0
:10257000D52F832F80CF80913C02811509F4B8CFED
:10258000E0903A02F0903B020E940B098E199F09DD
:10259000059708F4ADCF45E050E068E472E0C8016B
:1025A0000E947030892B41F085E0E8E4F2E0D80128
:1025B00001900D928A95E1F710923C0299CFC0905C
:1025C0003602D09037020E940B098C199D09843F76
:1025D000914008F0A0CF80913802811531F2F701C7
:1025E00085E011928A95E9F710923802A09139029C
:1025F000B0E0A35CBD4F85E0FE013B9601900D92DB
:102600008A95E1F7B2CF809135028F3F39F40E946D
:102610000B098093360290933702DDCF8F5F809352
:1026200035028A3008F491CFF2CF85E0F801AEE1AF
:10263000B2E001900D928A95E1F78EE192E00E945E
:10264000CA0780931D02C0902302D0902402E0901C
:102650002502F09026028091310290913202A091E1
:102660003302B0913402C816D906EA06FB06B1F06F
:10267000C0923102D0923202E0923302F0923402E0
:102680000E941A0AC61AD70AE80AF90AC092540226
:10269000D0925502E0925602F092570280912702A2
:1026A0000E947F0762CFA0E0B0E0E9E5F3E10C947F
:1026B000BB2FEC019881913000F109F044C0898171
:1026C000813051F48A81239660E570E0893311F0FE
:1026D00060E070E0B0DDEECF823021F48A81239695
:1026E000C2DCE8CF833021F48A81239654DDE2CF27
:1026F000843041F022968111DDCFCDB7DEB7E9E01D
:102700000C94D72F8A81239620E030E09AE0482F5E
:102710004053550B4A30510560F02115310559F3EE
:10272000EFE9FFE03197F1F700C0000021503109D7
:10273000F4CF929FB001939F700D11249A01260F40
:10274000371F8991E4CF2196E92FF0E0E458FD4F3F
:102750008491B82E292F26952695269530E0F901EB
:10276000E459FD4FE4909770F12C092E02C0F594C6
:10277000E7940A94E2F7F901E45AFD4FC490D12C92
:10278000092E02C0D594C7940A94E2F7245B3D4F0A
:10279000F901049110E002C0159507959A95E2F7AA
:1027A000E0FE02C081EE5FDCC0FE02C086EE5BDCB4
:1027B00060E070E08B2D3FDDC0FE02C086EEEBDCFA
:1027C000E0FE02C081EEE7DC00FF74CF60E070E065
:1027D0008CE280CFCF92DF92EF92FF921F93CF9344
:1027E000DF9300D000D0CDB7DEB7C0901902D090F3
:1027F0001A02E0901B02F0901C020E941A0ADC01EF
:10280000CB018C199D09AE09BF0911E084369105F1
:10281000A105B10578F10E94260ADC01CB010296E0
:10282000A11DB11D89839A83AB83BC838091220152
:1028300090912301835E9D4F20912101422F50E012
:10284000253008F044E09E012F5F3F4FB9010E9400
:102850007D3082E090E00E94442F182F811551F0C6
:102860000E941A0A6093190270931A0280931B0245
:1028700090931C02812F0F900F900F900F90DF917B
:10288000CF911F91FF90EF90DF90CF900895AF927E
:10289000BF92CF92DF92EF92FF921F93CF93DF937D
:1028A00000D000D000D0CDB7DEB75B0180E090E073
:1028B0000E94442F182F811509F45FC080911401E4
:1028C000482F50E0811141E060911501709116018F
:1028D000635E7D4FCE0106960E947D30C0902D0232
:1028E000D0902E02E0902F02F09030020E941A0A3F
:1028F000DC01CB018C199D09AE09BF098436910515
:10290000A105B10538F48EE192E00E94CA079E81CC
:10291000891799F181E090E00E94442F8115C1F15F
:1029200080911C01482F50E0863008F045E060910E
:102930001D0170911E01635E7D4FCE0101960E94C4
:102940007D308EE192E00E94CA079E81891320C0EB
:102950000E941A0A60932D0270932E0280932F0218
:102960009093300285E0FE013196A8E2B2E001903A
:102970000D928A95E1F781E00CC085E0EEE1F2E08E
:10298000DE01119601900D928A95E1F71111EACFBF
:1029900080E095E0E8E2F2E0D50101900D929A9591
:1029A000E1F70F900F900F900F900F900F90DF9125
:1029B000CF911F91FF90EF90DF90CF90BF90AF909D
:1029C0000895A1E0B0E0E7EEF4E10C94BC2F109183
:1029D000930210FF44C01695169516951983009121
:1029E0002702C0901502D0901602E0901702F090D6
:1029F00018020E941A0ADC01CB018C199D09AE094C
:102A0000BF0984369105A105B10510F4011711F134
:102A100080912A0190912B01835E9D4F2091290185
:102A2000422F50E0211141E09E012F5F3F4FB9013D
:102A30000E947D3083E090E00E94442F811559F080
:102A40000E941A0A6093150270931602809317026F
:102A50009093180281E02196E8E00C94D82F10E0C2
:102A6000BDCF86E090E00E949D308093930282FD6E
:102A700007C08DE38093930283E992E00E94930C58
:102A800080919302803420F0877088638093930252
:102A900090919302892F817090FF04C0892F8695B1
:102AA000869586950C94EE060F931F93CF93DF9334
:102AB000863008F56A30F8F44630E8F4C42FD0E0E8
:102AC000CC0FDD1F9CE0699FC00DD11D112498E73C
:102AD000899FC00DD11D1124CE0189960E949D3081
:102AE000082FCE018A960E949D30902FDF91CF91C2
:102AF0001F910F91089580E090E0F8CF462F20912C
:102B00005A0230915B02232B89F4703F39F4603F05
:102B100069F4809158029091590208957A3030F406
:102B2000663020F4863010F4672FBECF80E090E04E
:102B30000895CF92DF92FF920F931F93CF93DF936D
:102B40006C010091A8038091A703082BC5E0D0E099
:102B500010E0C8010C2E02C0959587950A94E2F703
:102B600080FD0CC02197A8F7F12C8F2DDF91CF911C
:102B70001F910F91FF90DF90CF900895FC2EB6012A
:102B80008C2FBCDF0E94EA05019761F3EECF1F9303
:102B9000CF93DF93FC012581C081D181CE01211526
:102BA00079F0611569F0C5DF182F682FCE010E94FA
:102BB0001504BE01812FA2DFDF91CF911F910895EF
:102BC0000E944B04182FF5CFCF93DF93EC01B1DFB8
:102BD000BE0194DF0E94EA05DF91CF910895FC01C8
:102BE0002481211599F080819181EEDF282F929523
:102BF0009F70963099F060F4925F9F70923030F43D
:102C0000203FB1F038F481E0283E38F080E00895AC
:102C10009A5FF3CF81E0243FC9F7089591E0213F07
:102C200009F090E081E0283E08F080E0892B0895CB
:102C300081E00895673671058105910528F4CB017F
:102C400087569C4F0C949D3080E0089585E290E07B
:102C50000E949D30863A69F486E290E00E949D30A1
:102C6000823339F487E290E00E949D3091E0853E06
:102C700009F090E0892F81700895AAE0B0E0E3E4C4
:102C8000F6E10C94B72FC0901202D090130281E0AD
:102C90008093120210921302812C912CE12C54018A
:102CA000F12C15C0F80125913591472D6F2D8E2DF2
:102CB0000E94AF0C0E5F1F4F7394872D863091F7E3
:102CC00086E0A80EB11CF3948F2D8A3039F085016F
:102CD000000F111F04501D4F712CE4CFE3948CE3BF
:102CE000880E911C8E2D8630D1F619821A821B8295
:102CF0001C821D821E821F82188688EC89871A8694
:102D000009EF12E07E018FEFE81AF80A4AE050E07E
:102D1000B801C7010E94D730065F1F4F5701093421
:102D200083E0180799F7F70189E011928A95E9F78E
:102D30008FEF9FEF8D839E8387E08A874AE050E084
:102D4000B801C5010E94D730065F1F4F093983E0E3
:102D50001807A1F7C0921202D09213022A96EDE052
:102D60000C94D32FAAE0B0E0E8EBF6E10C94BE2F70
:102D70000AE912E089E4E82E83E0F82E4AE050E008
:102D8000B701CE0101960E948D30F801389687E098
:102D900011928A95E9F789819A81F801808391835C
:102DA0008F8182838D8183838885848389858583D0
:102DB0008B819C81868397838A8587FD04C02BEE57
:102DC00031E02587368780FF03C0F80191E09087C6
:102DD00081FF04C0F80190859260908782FF04C053
:102DE000F80190859460908783FF04C0F801908576
:102DF0009860908784FF04C0F80190859061908767
:102E000085FF04C0F8018085806280878AE0E80E33
:102E1000F11C015F1F4F89E9E81683E0F80609F00D
:102E2000ADCF2A96E6E00C94DA2F9B01883070F43F
:102E30009AE0899FB001112467507D4F4AE050E02D
:102E4000C9010E948D3080E090E008958FEF9FEFE0
:102E50000895AAE0B0E0EFE2F7E10C94C22F392F19
:102E6000375561F4BE016F5F7F4FDFDF892B31F48F
:102E700089859A852A96E2E00C94DE2F88EC90E012
:102E8000F9CFA0E0B0E0E7E4F7E10C94BD2F7B01BF
:102E9000C42FD22FD02E8115A9F04093A1030E94F8
:102EA0000B098093E9019093EA0181E0C1FD84E080
:102EB000C0FD880FC2FD8295D4D9CDB7DEB7E7E05B
:102EC0000C94D92F8091A103481336C00091E901D9
:102ED0001091EA010E940B09801B910B8C01C70124
:102EE000B8DF0817190740F51D2F105ECD17A1F0A8
:102EF0008C2F8770C1E09C2F01C0990F8A95EAF74B
:102F0000892FB5D9183040F48D2F877001C0CC0FB0
:102F10008A95EAF78C2FA5D960E070E08D2D8BD9CA
:102F200081E0D1FD84E0D0FD880FD2FD829518307C
:102F300008F0C3CF9CD9C1CF81E0C1FD84E0C0FDC2
:102F4000880FC2FD8295F6CFA9E0B0E0EAEAF7E18A
:102F50000C94B22F7C01FC018481811509F4E6C038
:102F600061E0C70114DE8C01F7018581811529F12B
:102F7000E0919D03F0919E033097F9F00E171F0723
:102F8000E1F08E2F887F90E0892B09F080C0F0E07F
:102F9000E295F295F07FFE27E07FFE27E35EFC4F8F
:102FA00085818460858300831183CF01F6D91092D7
:102FB000A90361E0C701EBDD8C01003482E518074D
:102FC00009F477C008F066C0043282E5180709F4F6
:102FD0008FC0053282E5180709F492C0033282E5FA
:102FE000180709F474C0F7018581811509F46EC1D1
:102FF000C80197578038910508F01AC1003208F0CF
:1030000086C066E670E080E090E014DE81117FC04B
:10301000A12CB12C4501011191C08E010F5F1F4FF2
:10302000F80184E011928A95E9F7B401C50102DE46
:103030008983811509F46BC0240135019FEF491A7A
:10304000590A690A790A8130F9F4B201C301F2DD43
:10305000D82E8A83811509F45AC0B401C5016E5F68
:103060007F4F8F4F9F4F2D2D2150233008F07BC075
:1030700023E0820E911CA11CB11C24013501DADD74
:103080008B83811509F49AC0C8010DDB97C0E0E07D
:10309000F0E086CF013482E5180799F0023482E52A
:1030A000180709F0A0CFF7018581811581F182E031
:1030B00005C0F7018581811551F180E00E94810CE6
:1030C00026C0F7018581811511F181E0F7CFF70165
:1030D0008581811549F083E00E94010445E064E0A8
:1030E00083E00E947E0413C083E00E940A04F6CFAE
:1030F000F7018581811511F084E0EECF84E0F5CFF2
:10310000F70185818115B1F085E00E94010480916D
:10311000AA03877059F0F7018581811539F08091F4
:10312000F10382FF03C082E00E94C5042996E2E118
:103130000C94CE2F85E00E940A04E9CF87E688161A
:103140009104A104B10419F3B401C50173DD9FEF2B
:10315000891A990AA90AB90A8111F0CF01505BCFE7
:103160002B013C012BC02D2D2550233080F524014F
:10317000350123E0420E511C611C711C5BDD8B8309
:103180008115E1F084E0880E911CA11CB11CB201F4
:10319000C30150DD8C83811579F08B819C81813056
:1031A0002FEF920710F0982F80E02D2D263049F058
:1031B000273051F00E94552424013501420153016A
:1031C0002FCF0E940624F8CF0E942524F5CF2D2D65
:1031D000243031F62FDDD82E811509F498CFB401B3
:1031E000C5016D5F7F4F8F4F9F4F24DD811509F41F
:1031F0008ECF94E0890E911CA11CB11C24013501D5
:10320000282F2150330B4FEF429FC001439F900D59
:1032100011242D2D2150330B820F931F009771F233
:103220000197EFE9FFE03197F1F700C00000F6CF1A
:10323000033088E7180709F4AAC068F5013088E769
:10324000180709F4A2C0023088E7180709F4CEC0B5
:10325000011588E7180709F490C0023A82E51807BB
:1032600009F068C021EE30E0277081E001C0880FCE
:103270002A95EAF7482F2091970230919402311550
:1032800009F401C1F7013581311509F4F7C0282B84
:10329000209397023CCF043088E7180709F487C0D1
:1032A000053088E7180709F4B3C003378CE718071F
:1032B000A1F6F7018581811509F429CF8091940247
:1032C000811509F4B7C00E94501121CF680189EA25
:1032D000D80E59F769E872E08C2DA7DD892B29F506
:1032E000C60182959295907F9827807F9827FC0150
:1032F000E35EFC4F2281213071F5209189023091EB
:103300008A02232B91F020918B0230918C02232B87
:1033100061F020918D0230918E0240918F02509188
:103320009002242B352B232BF1F0F7018581811599
:1033300009F493CF033A82E5180708F08BC0C8015F
:103340009052903208F48DC0013E110509F48ACFE5
:10335000053E110582C0223041F720918D02309147
:103360008E02232B11F3FC01EE5DFC4F20812E7F9A
:103370002083835E9C4F11D8D8CF87E00E947F07BF
:1033800083E992E00E94930CC2CE80E0F7CF809157
:103390009302883028F188508093930291E088301E
:1033A00008F490E08091930290FB80F913C0909113
:1033B0009302892F869586958695983340F48F5F82
:1033C000880F880F880F9770892B809393028091C4
:1033D000930281608093930283E992E00E94930CB0
:1033E000809193028695869586950CC08091930274
:1033F00080FF0BC08E7F8093930283E992E00E944E
:10340000930C80E00E94EE0682CE0E94990C7FCE43
:10341000809193028695869586958F5F8F7188300F
:1034200008F080E0880F880F880F909193029770C2
:10343000892BB2CF1092A5030E94ED040E940B09C4
:1034400088579C4E809395029093960281E08093DA
:1034500094025DCE023B82E5180721F525EE30E0AF
:1034600003CFF70186818031E8F4812F8F7190E0DE
:103470008230910509F4F6CE4297EFCF80958223F2
:103480008093970244CE322F342361F0982F909589
:103490009223909397020E94E504F701858181159C
:1034A00009F435CE80919402811509F460C0D09062
:1034B000A503C090A4030E940B0988579C4E8093DB
:1034C000950290939602F7018581811509F44FC00A
:1034D0008C2D8D298D7909F07CC01035D8F41034ED
:1034E00008F07EC0063E110509F441C0C8019052A3
:1034F000903208F07AC08681803108F462C0802F53
:1035000090E01092A9038D329105E9F482E0809356
:10351000A9036FC0003E82E5180708F045C0003CD3
:1035200082E5180720F5003A82E51807E0F4003636
:1035300082E51807E0F4C801925580349105B8F08F
:103540001092A903C8018E32910508F05FC088323D
:10355000910508F04CC08E31910508F04AC00497DF
:103560004A97A0F236C0043B82E5180749F7F701F5
:103570003580311409F454C00E358CE7180709F46E
:103580004BC00F358CE7180749F00D358CE718074D
:1035900009F046C0809131018115F1F1109231019D
:1035A00080E00E945911B3CD09378CE7180728F441
:1035B00007378CE71807D8F6C3CF0B378CE7180707
:1035C000D5CF812F8F71843191F2863111F4109211
:1035D000A9030E945011809197020E94DF04C7CF77
:1035E0008681803108F08BCFC2CFC8018ACF8A97FD
:1035F00081F780919702811531F08091A90392E0C3
:1036000089278093A9030E94EC0CB1CF8C349105DB
:1036100081F38D329240ECCF81E08093310177CD00
:1036200080913101811166C0912F975509F0FBC03F
:10363000A02E88EFA822B12CA114B10409F067CD07
:10364000E02FF0E0E295F295F07FFE27E07FFE2785
:10365000CF01835E9C4F6C01D70115968C91EE5D76
:10366000FC4F908180FB90F99083811509F4D6C1BD
:103670000E940B0980939F039093A003F60182811F
:103680008F5F82838091A9039091A503892B838307
:103690008091A40384834681578166857785C6011E
:1036A0000E947B08F601858181FF5801A0929D034D
:1036B000B0929E03F7019581911509F4F0C510921F
:1036C000A103980130572332310508F0F6C584E094
:1036D00090E00E94A5308093F0039093F103F801ED
:1036E000E150F047E232F10508F0DFC1E35FFE4C44
:1036F0000C945030480180EE881A91089091A603EE
:103700008091A503982B8091A403982B9D8388E03A
:103710008816910408F05AC09801277081E001C012
:10372000880F2A95EAF7311409F44BC02D81282B14
:103730002D83F701808191810E944B0421E030E0CC
:1037400002C0220F331F8A95E2F7290180911303EB
:10375000909114038E839F8380911B0390911C038F
:10376000888799876AE9C62E62E0D62EA12CB12CF3
:103770008D81811104C0F6018281811117C0F6018B
:10378000838190E08421892B89F08085982F977020
:1037900009F487E098E08916910408F068C03114B4
:1037A00009F461C086958170811166C08FEFA81AF7
:1037B000B80A8FE0C80ED11C88E0A816B104C1F683
:1037C0001EC080959D8198239D83B3CF311038C052
:1037D00080911B0390911C030817190781F4109224
:1037E0001B0310921C0310921703109218031092DF
:1037F000190310921A031092150310921603809168
:10380000130390911403009709F40ECF28E0821659
:10381000910408F0EDC06D810E94E307811103C09F
:1038200081E00E945911F7018581F801E851FC47B8
:10383000E730F10508F03ECFE15DFE4C0C945030CE
:1038400000931B0310931C030E941A0A6093170332
:10385000709318038093190390931A031092150321
:103860001092160366CF82FB882780F99DCF311412
:1038700009F49CCF80FF9ACFF60160807180061515
:10388000170519F4311409F491CF8E819F818C159D
:103890009D0509F48BCFF6010584F685E02D309760
:1038A00021F08081811509F481CF6D81C6010E94CC
:1038B000E307811509F47ACF81E00615170509F0B1
:1038C00080E08321282E6114710441F0811106C02B
:1038D000888599856816790609F068CF80E00E948E
:1038E0005911C0921303D092140381E08093120304
:1038F0008FE08A9DF0018B9DF00D1124E656FD4F5F
:1039000085818093990221100EC06114710459F0D1
:10391000808191819C0124503109213A310508F0C0
:103920004AC00E94FC088FE08A9DF0018B9DF00D3B
:103930001124E656FD4FC680D780C60191509F31B5
:1039400010F480EED82277247394C60101978F3348
:103950009E4708F0712C8FE08A9DD0018B9DB00DA1
:103960001124A656BD4F1996ED91FD911B973097E6
:1039700041F01B966D917D9181E00995972D9823DB
:10398000792E7114A9F08FE08A9DF0018B9DF00DC6
:103990001124E656FD4F868197810E94C4038093CF
:1039A000980288E08816910448F4C6010E94410AF2
:1039B0000E94EC0C0BC00E94CB10B5CFC60104973F
:1039C000813A910548F48C2D0E94E208211409F4F3
:1039D0002BCE0E94EC0C9BCB0E94EC0C8FE39CE95D
:1039E0000197F1F700C000008C2D0E943310EECF3C
:1039F000FC01208131810217130741F4311009C005
:103A00001092120380E00E9459110ECE311409F475
:103A10000BCEFC01808585FD07CEF4CFF6014485F1
:103A2000558566857785C6010E947B08F6018581EC
:103A300081FF40CEC6010E94B21180919D039091FA
:103A40009E030817190709F035CE10929D031092B6
:103A50009E0330CE06E221EE41EE6AE17CE711DA08
:103A600056CB07E225EE45EE6BE17CE7F8CF06E2A8
:103A700021EE40EE68E17CE7F2CF07E225EE44EE6E
:103A800069E17CE7ECCF06E221EE42EE6CE17CE7F7
:103A9000E6CF07E225EE46EE6DE17CE7E0CF08E2F7
:103AA00021E045EE6EE17CE7DACF8091F0038160A2
:103AB0008093F0036091F0037091F10384E090E053
:103AC0000E94D3300E94400D22CB8091F103886088
:103AD0008093F103EFCF8091F0038260E9CF809172
:103AE000F0038460E5CF8091F0038860E1CF80919E
:103AF000F1038160EDCF8091F1038260E9CF809185
:103B0000F0038061D5CF8091F0038062D1CF8091A6
:103B1000F0038064CDCF0E94400D8091F003806857
:103B2000C7CF8091F0038C60C3CF8091F103836095
:103B3000CFCF8091F0038E7FBBCF8091F103877F41
:103B4000C7CF8091F0038D7FB3CF8091F0038B7F3F
:103B5000AFCF8091F003877FABCF8091F1038E7F51
:103B6000B7CF8091F1038D7FB3CF8091F0038F7E2B
:103B70009FCF8091F0038F7D9BCF8091F0038F7B4F
:103B800097CF0E94400D8091F0038F7791CF809165
:103B9000F003837F8DCF8091F1038C7F99CF90913B
:103BA000F003892F8B7F92FF8460877F92FF88606C
:103BB0007FCF8091F103982F909590FB80F990FB37
:103BC00081F986CF9091F003892F8F7B96FF8064D7
:103BD0006FCF0E94400D9091F003892F97FB87F9DA
:103BE000805866CF61E08EE090E00E94B93062CFED
:103BF00060E0F9CF9091F003892F8F7E94FF806170
:103C000057CF9091F003892F8E7F90FF816050CF26
:103C10009091F103892F877F93FF886059CF89E2C4
:103C20005EC389E247C307378CE7180779F0083786
:103C30008CE71807A1F09801205E3245203231054B
:103C400098F4911111C0802F8F7138CA81E09115BD
:103C500041F00E94010443E062E081E042CA82E058
:103C6000F6CF0E940A04F7CF4091A3038091A803E6
:103C7000282F20953FEF70E02423372321153105AD
:103C800019F048234093A3030B372CE7120741F4A4
:103C9000911509F43CCA0E94E9030E94030837CA3F
:103CA000003482E5180708F04CC0003282E518079E
:103CB00008F04EC0103540F5103408F05CC0911586
:103CC00009F470C00A358CE7180709F4D2C008F06F
:103CD000B7C001308CE7180709F4C9C003308CE77E
:103CE000180709F4BEC001151C4709F05BC00E940B
:103CF000400D8FEF94E32CE0815090402040E1F79D
:103D000000C000000E94FE0B980130553230B8F61A
:103D1000980145E0369527954A95E1F7822F8F70F7
:103D20002091A30330E041E0082E01C0440F0A9423
:103D3000EAF72423232B19F29111AFCF1092A50398
:103D400048CE9801205C32452032310508F0B7CFCB
:103D5000802F8F712091A30330E041E0082E01C035
:103D6000440F0A94EAF72423232B09F4A8CF9115D2
:103D700009F4CDC992CFF7018681803108F09FCF39
:103D8000911110C0212F2F7081E090E002C0880FA8
:103D9000991F2A95E2F72091A30382239323892B6D
:103DA00009F0B5C9F701858100811181811509F4F8
:103DB00064C0C8010E949915D82E682FC8010E94BE
:103DC0001504B8018D2D0E947E150E94EA05182F5A
:103DD000A92EF701C580B680B2948FE0B8228091F9
:103DE000AA03877001F1DC2CC114F1F0892F807FC8
:103DF000803461F0812F805E8830A8F0892F807E2A
:103E0000803221F4123078F0B11469F08091F1031E
:103E100082FF09C082E00E94C5048091AA038770D6
:103E2000DD24D3948111D12CEA2DE295EF708A2DF7
:103E3000803C08F07DC0F0E0EA5CFE4C0C94503011
:103E40000B358CE71807B9F00C351C4709F0AACFE1
:103E50008091F103002482FF0394802D0E94D50CF1
:103E6000A1CF6FEF7FEF80E090E00E94D3300E94FF
:103E70005E0D81E0F3CF80E0F1CFC8010E944B04DA
:103E8000D82E9FCF0A2D0F70803110F00295007F41
:103E9000C114A9F0011559F0812F805E883010F00F
:103EA000111107C0802F0E94DF040E94EC0C812FAB
:103EB0003DC08091A903802B8093A903F6CF812F69
:103EC0000E94CB100115A1F1812F805E883010F087
:103ED000111104C0802F0E94E50406C00095809156
:103EE000A90380238093A9030E94EC0C21C00A2D12
:103EF0000F70807F803211F00295007F113040F00A
:103F000009F481C0C11409F48CC0B114A1F1CFCF60
:103F10008091F10382FD2BC0C11419F1011529F024
:103F2000802F0E94DF040E94EC0C80E00E9433107E
:103F3000D11409F4D5C08091AA0380FDD1C0F70146
:103F400015828695869586950E940104C7010E9478
:103F5000A4178091AA038695869586950E940A04E7
:103F6000BFC080E00E94CB10011511F3B3CFC11484
:103F700069F1B11004C0802F0E943111D9CF8B2D6F
:103F8000813089F48091A403182F8023081781F2CF
:103F90000E940B098093AD039093AE03812F802B79
:103FA0008093A403C5CF853019F6802F0E9431116C
:103FB000802F0E942A098091A603902F9823091729
:103FC00009F4B6CF802B8093A603B2CFB11011C0F5
:103FD000802F0E943711802F0E942A098091A6030A
:103FE000902F982309F4A4CF009508230093A603EB
:103FF0009FCF8B2D813009F09BCF8091A50380232B
:1040000009F496CFE5CF8B2DC11421F0863008F04E
:104010008FCFB1CF853008F08BCF802F0E94371122
:1040200087CFB114D1F3193349F48FEF97EE23E022
:10403000815090402040E1F700C00000812F0E9495
:10404000CB1076CF869586958370813060F009F02D
:104050006FCF812F9A2D9370C11002C080E090E045
:104060000E94BB0865CF812F9A2D9370C11002C0AA
:1040700080E090E00E9494085BCF6C2D812F0E941D
:10408000630956CF8370E1F5C11028C0812F829556
:1040900086958770880F880F412F4F70082E01C0BA
:1040A000440F0A94EAF7212F207114FF06C02FE075
:1040B00001C0220F8A95EAF720958A2D869586956C
:1040C0008370982F8230A1F08330B9F08091A703DC
:1040D000913059F0242B82230E94FB030E94810817
:1040E00060E0C7010E94C71521C8842B822BF4CF42
:1040F000242B8091A7038227EFCF822F842BECCF34
:10410000C11459F1A0FEEACF812F82958695877060
:10411000880F880F412F4F70082E01C0440F0A945A
:10412000EAF7212F207114FF06C02FE001C0220FF3
:104130008A95EAF720958A2D869586958370982F23
:10414000823091F08330A9F08091A803913049F03A
:10415000242B82230E94FE03C1CF823008F4BECFFD
:10416000D3CF842B822BF6CF242B8091A8038227D8
:10417000F1CF822F842BEECF8F70082FC11431F036
:104180000E940104812F0E943111A8CF812F0E942B
:104190003711802F0E940A04A1CF123F81F170F4E1
:1041A000103FC9F0113F91F0C11409F467C0B11478
:1041B00009F461C0812F0E94331090CF133F29F181
:1041C000143F91F78091F10382FD2CC08A2D8F71ED
:1041D000C11401F317C08B2DC11479F0853008F09C
:1041E0007DCF8A2D8F71282F81E001C0880F2A95FD
:1041F000EAF79091A8038927ADCF8630F0CF8F7171
:10420000C110C8CF0E94010469CF80E0C11409F435
:10421000A1CF8A2D8F71982F81E001C0880F9A95C8
:10422000EAF798CFC114C1F08091AA038770843057
:1042300049F41092AA031092AB031092AC038A2D9A
:104240008F71A8CF8B2D63E0853008F047CF8A2D82
:104250008F710E94170942CF8B2D853040F010924C
:10426000AA031092AB031092AC0364E0F0CF81E09C
:104270000E94C50433CF8A2D8F71C4CFB114F9F2D7
:10428000193349F48FEF97EE23E08150904020409E
:10429000E1F700C00000812F0E94CB101FCF063134
:1042A0008CE7180709F0BFCC8091A203811509F4AF
:1042B000B8CC85E30E94FC088CCB06318CE718074C
:1042C00009F0B1CC8091A5038A7A91E0811101C0F7
:1042D00090E09093A203811509F4A1CC85E30E949C
:1042E000E20877CBEF92FF920F931F93CF93DF9368
:1042F0008091EF03803108F047C08091EE03811573
:1043000009F442C08091B0039091AF039817E1F196
:104310007C0197E0899FE0011124FE01EF54FC4FDE
:1043200084818115B1F191818091EA03981331C0A4
:1043300090818091E90398132CC08581811129C057
:10434000028113818091EB039091EC03081B190B00
:1043500060E089EE93E00E94C7150E9429170817B4
:104360001907B8F48091EF038F7080618093EF0399
:10437000C954DC4F88818F708061888389EE93E017
:104380000E94A4170E94BB04CDB7DEB7E6E00C94F0
:10439000DA2FC70183958770B7CFADE0B0E0E3EDCA
:1043A000F1E20C94B52F8C0186E0F801DE0118963D
:1043B00001900D928A95E1F7F801F580E48089EE8D
:1043C000882E83E0982E8091ED03811117C0E114AF
:1043D00091F0F11409F4B3C0C8010E94EF158115E2
:1043E00009F4ADC087E0F801A9EEB3E001900D92A9
:1043F0008A95E1F777DFFF24F39462C0C280D3800F
:10440000B090EE038091EB039091EC033601681AB3
:10441000790AB11409F4DFC08081582E8181A82E59
:1044200060E089EE93E00E94C7150E942917681684
:10443000790608F088C0E114F1F28091EA03F801EE
:104440009181E090EF032E2D203108F05AC098138F
:1044500016C09091E9038081981311C0F1104BC0F0
:104460008E2D8F7080618093EF0389EE93E00E9420
:10447000A4178091EF03F8018683F12C21C0F1107D
:104480003AC040E06A2D852D0E949C0440E06A2DD0
:10449000852D0E949C04F82E8111EFCF8885998587
:1044A0000E94E415292F22952F70903470F49F708C
:1044B0002230A0F09115B1F0F8019681903190F47E
:1044C0008F2D2D96EFE00C94D12F2A5F2F70223084
:1044D00068F0C8010E94A417FB2CF2CF911511F0CF
:1044E000811571F3805E883058F3F3CF803F40F33D
:1044F000815F8330F9CF8091EF0381608093EF0378
:10450000BCCF981314C09091E903808198130FC019
:10451000F1100DC0E682C8010E94A41787E0F801DF
:10452000A9EEB3E001900D928A95E1F764CFC8013E
:104530000E94EF15811519F08E2DF11035C0C801BC
:104540000E94A41758CFB090EF038B2D803150F408
:1045500089EE93E00E94A417F40187E011928A95F6
:10456000E9F78BCFE11409F446CF9091EA03F80103
:104570008181981311C09091E903808198130CC038
:10458000F1100AC0B682C8010E94A417F40187E0A6
:1045900011928A95E9F72FCFC8010E94EF15811576
:1045A00071F2F11461F28B2D803208F41BCF8091EF
:1045B000E9039091EA0389839A83CB82DC8280911C
:1045C000ED038D831E828091EF038F83CE010196D0
:1045D0000E94A41707CF60E089EE93E00E94C71500
:1045E0000E9429176816790608F0B6CFE11409F47D
:1045F00002CFF11409F4A3CF9091EA03F80181816D
:10460000981324C09091E903808198131FC0809172
:10461000EB039091EC03C81AD90A88ECC816D104B0
:1046200008F07CCF9091EF0390FD78CF903108F4A3
:1046300075CF892F9683907F903F09F46CCF982F88
:10464000907F905F8F70892B868365CFC8010E9411
:10465000EF158111C7CE8091EF0381608093EF0346
:104660006ECFABE1B0E0E7E3F3E20C94C02F4E8BEA
:104670005F8B688F798F8A8F192F9B8F9111109282
:10468000A9031D8A86E0FE017696DE011F96019041
:104690000D928A95E1F70A8D8091F10382FF1FC088
:1046A0000E940B092091AB033091AC03821B930B4A
:1046B0008838934138F08091AA0382FD03C082E0DC
:1046C0000E94C5040E940B092091AD033091AE03F6
:1046D000821B930B8838934110F00E94ED04011562
:1046E00061F00B8B1C8B61E0CE010F960E94C71509
:1046F00061E0CE010F960E94C7150B8B1C8B87E0E3
:10470000FE013F96DE01189601900D928A95E1F721
:10471000CE01089642DE811128C02091AF0330916E
:10472000B00387E0AE01485F5F4FFA01475051097F
:10473000DA0101900D928A95E1F78C858115A9F037
:10474000822F90E08395877090E0AC0134171506B6
:10475000B1F40E94400D1092AF031092B003E9EE45
:10476000F3E087E011928A95E9F78091B003909188
:10477000AF03891317C06B96E4E00C94DC2F97E02D
:10478000929FD0011124AF54BC4F9E012F5F3F4F29
:10479000F90101900D929A95E1F74093AF030E94C1
:1047A000BB04E3CF27E0829FC00111248F549C4FAC
:1047B000F4DD811501F38091B0039091B10301966E
:1047C00087708093B003D1CFA6E0B0E0EAEEF3E2C9
:1047D0000C94C02F0E940B098C0180915C02909177
:1047E0005D028017910771F019821A820E940B09ED
:1047F000BC0149815A8180E090E033DF00935C0284
:1048000010935D022696E4E00C94DC2FA6E0B0E065
:10481000ECE0F4E20C94C22F80935802909359027A
:10482000903230F40E94B6102696E2E00C94DE2F0F
:1048300080EF89838A830E940B098160BC014981D2
:104840005A8181E091E00DDFEFCFA6E0B0E0EBE22E
:10485000F4E20C94C02F8C018093580210935902FB
:104860001032B0F4802F0E94CB10C801805E9109F5
:10487000089728F066E471E10115110511F467E36A
:1048800071E1C8010E94E0032696E4E00C94DC2F5D
:1048900080EF89838A830E940B098160BC01498172
:1048A0005A8181E090E0DDDEEFCFCF93DF93EC0122
:1048B000ADDFCE01CADFDF91CF9108950F931F9333
:1048C000CF93DF938C01862F69E872E00E94151761
:1048D000892B91F4C0918902D0918A02209761F0CE
:1048E000F8018281833039F4CE01DFDFCE01DDDFD4
:1048F000CE01DBDF01C0E0F7DF91CF911F910F9177
:1049000008950F931F93CF93DF938C01C62F69E80F
:1049100072E08C2F0E941517892B09F058C0EC2FDC
:10492000F0E0D80112968C911297E451FE4F81303D
:10493000A9F415968C9182FD4FC080FF4DC082E096
:10494000808380918B0290918C020097C1F48091BA
:10495000890290918A020097D1F111C08230A9F5A5
:10496000D80115968C9182FD26C080FD0AC083E097
:10497000808380918D0290918E020097F1F046DF46
:1049800026C084E0808380918F02909190020097EE
:10499000B1F78091890290918A02009701F185DF39
:1049A00080918B0290918C02009749F78091890247
:1049B00090918A02E4CF85E0808380918902909172
:1049C0008A02009721F071DFF1CF86E08083DF91CA
:1049D000CF911F910F91089581E08083B8CF80918E
:1049E0008B0290918C02B7CF0F931F93CF93DF93DD
:1049F0008C01C62F69E872E08C2F0E941517892B55
:104A000071F4D0E0C451DE4F8881F801128218821F
:104A10008330E9F048F4813059F0823081F0DF9141
:104A2000CF911F910F9108958430B1F08530B9F77F
:104A30008091890290918A02009789F306C0809143
:104A40008B0290918C02009799F3FFDEE8CF809162
:104A50008D0290918E02F7CF80918F0290919002FB
:104A6000009799F72091890230918A0280918B02F8
:104A700090918C0221153105F9F2009731F7C901A7
:104A8000E4CFA0E1B0E0E7E4F5E20C94B42FFE013E
:104A90003196DF0180E11D928A95E9F707E010E089
:104AA00099E9A92E93E0B92E612C712C23014A18A3
:104AB0009E2E8F2E6201730181E14816510461041C
:104AC00071041CF080E1C82ED12CA601B501892DFE
:104AD000982D0E94AA30AC0CBD1C0D2C000C0008B7
:104AE0004C185D08600870080150104019F7609676
:104AF000E0E10C94D02F6FEF85E290E00E94B93096
:104B00006FEF86E290E00E94B9306FEF87E290E0AD
:104B10000E94B93060E088E290E00E94B9300E94C3
:104B20003D16AFDF66EA85E290E00E94B93062E3AD
:104B300086E290E00E94B93065EE87E290E00C9446
:104B4000B930CDB7DEB7E0970FB6F894DEBF0FBE31
:104B5000CDBF85B7806885BF85B7806885BF84B7BE
:104B6000877F84BF0FB6F894A89580916000886114
:104B700080936000109260000FBE80E890E00FB656
:104B8000F89480936100909361000FBE81E0809360
:104B9000030186ED96E08093C4019093C5010E94C5
:104BA000B2070E94B2160E94AD0B0E945E0B80916C
:104BB000E20084608093E200789480911402811571
:104BC00099F08091E9001091EC008F7010FB112793
:104BD00017F9182B1092E9008091E80083FD0E94DC
:104BE000730D1F701093E90082E084BD93E095BDC2
:104BF0009AEF97BD80936E00109254021092550266
:104C000010925602109257020E942616811101C07E
:104C100072DF8091D80080618093D8008AE18A9504
:104C2000F1F700C08091D900182F117080FD04C0E9
:104C30000E94AD0B109214021093520255985D9889
:104C40008FE891E00197F1F700C0000088274D99A7
:104C500083958093530280930401809152028111C5
:104C60000E94632E809104018091040190E08111E3
:104C700001C095E09093470285E0891B809339023B
:104C80007CE4E72E71E0F72E01E511E0F701819158
:104C90007F018F3F11F00E94D8060E151F05B1F756
:104CA00001E511E0F80181918F018F3F11F00E9421
:104CB000D80681E007351807A9F7EDE3F2E08AE0AE
:104CC00011928A95E9F7E8E4F2E08AE011928A9578
:104CD000E9F780E090E00E94A530833E9E4F21F4EA
:104CE0000E942616811136C063EE7EEF80E090E0D0
:104CF0000E94D33060E082E090E00E94B93081E011
:104D00008093A70361E083E090E00E94B93060E007
:104D100074E184E090E00E94D3301982CE010196C4
:104D20000E94930CE8DE0E94990C85E00E947F07A8
:104D300083E992E00E94930C60E070E0AB018FE0A9
:104D400090E00E94CB3060E070E0AB0183E190E046
:104D50000E94CB3082E090E00E949D308093F6016B
:104D600084E090E00E94A5308093F0039093F103DB
:104D70000E94F2118FEF96E721E081509040204091
:104D8000E1F700C000000E94F21180913D0280FF17
:104D900008C06FEF7FEF80E090E00E94D3300E9468
:104DA000FE0B83E090E00E949D300E94FB03259A59
:104DB0002D9882E88093800089E1809381008FEFB5
:104DC0009FEF90938700809386000E9431150E9488
:104DD000311580915202811101C078D785E091E0B0
:104DE00080935E0290935F0210E41E018FEF281AF9
:104DF000380A80911402853059F48091140285306C
:104E000009F453C00E94400D0E9431150E94810890
:104E10000E94F21157EFE52E51E0F52E6DE3662E5C
:104E200062E0762EF301D7019D91808121E032E08E
:104E30002A173B0709F471C031969817A9F390908F
:104E4000520200E088248394F301D1903F01F701DE
:104E5000A1907F01AD1419F1AD24C12CBB24B394F2
:104E60008A2D8B21A9F0911499F0C9820A830E949E
:104E70000B098B839C838D8291E08D2D8B2109F40E
:104E800090E09E8349815A816B817C818D81E9DB31
:104E9000C394BB0C8C2D863019F7F701D2920F5FAB
:104EA0000A3091F60E94260A3BC080911402843099
:104EB00031F180E00E947F071092F40188E190E0D8
:104EC0000FB6F894A895809360000FBE1093600011
:104ED00083B7817F846083BF83B7816083BF789409
:104EE000889583B78E7F83BF0FB6F894A89580917D
:104EF0006000886180936000109260000FBE0E9485
:104F0000F211EDE3F2E080818111F7C4319687E47C
:104F100092E08E179F07B9F770CF981390CF54DCAB
:104F200080915202811509F478C0E0901503F09049
:104F30001603E114F104A1F180900502909006029D
:104F4000A0900702B09008020E941A0ADC01CB016F
:104F500088199909AA09BB094091010250910202DE
:104F6000609103027091040284179507A607B707A2
:104F7000B8F0C7010E94B6101092150310921603E4
:104F80001092050210920602109207021092080277
:104F90001092010210920202109203021092040277
:104FA000C0909D03D0909E03C114D10429F1A0901C
:104FB0009F03B090A0030E940B098A199B097C01F2
:104FC000C6010E9429178E159F05B0F480919D039C
:104FD000282F287F30E0232B09F030C190E0829504
:104FE0009295907F9827807F9827835E9C4FFC0145
:104FF000258122FF0E94CD1180919402811569F0D4
:105000000E940B092091950230919602821B930B0E
:105010008F3F9F4710F40E94501186E0E3E8F2E0D2
:10502000D10101900D928A95E1F7A0908402C09081
:10503000850200918602B0908702D090880210927B
:105040008502109286021092870210928802802FA9
:105050008C2909F441C0E0900B02F0900C020E94F0
:105060000B098E199F099C0190918102911509F4F9
:105070003FC42531310580F19F3F19F09F5F909328
:105080008102C11459F00E94360891E01C140CF002
:105090009FEF899F802D112480938502011559F07F
:1050A0000E94360891E010160CF09FEF899F802D2A
:1050B00011248093860280918502811569F0F09019
:1050C0008602F11449F00E942808809385028F2DF2
:1050D0000E942808809386028B2D8D2909F441C0F7
:1050E000E0900902F0900A020E940B098E199F09B4
:1050F0009C0190918002911509F4F5C32135310589
:1051000080F19F3F19F09F5F90938002B11459F096
:105110000E94560891E01B140CF09FEF899F802D90
:10512000112480938702D11459F00E94560891E00F
:105130001D140CF09FEF899F802D1124809388020D
:1051400080918702811569F0F0908802F11449F08E
:105150000E942808809387028F2D0E942808809340
:105160008802809184028A1119C08091850281157C
:1051700011F08C1113C020918602211511F020131B
:105180000DC090918802911511F09D1107C03091CA
:105190008702311103C0822B892B11F00E943B0939
:1051A00086E0F101A3E8B2E001900D928A95E1F763
:1051B0000E94810890910D02891721F080930D02C1
:1051C0000E941A0A80911402843009F012CE83E002
:1051D0008093E9008091E80082FF0BCE8091E80087
:1051E00090E085FF09C00E942D0B30E2C32ED12C28
:1051F0007101811589F191E08091E8008B778093AE
:10520000E800911509F4F5CDE0905A02F0905B02A8
:10521000E981E114F10471F1EE3F09F04DC08A819A
:10522000833020F08550833008F046C0EA81EE30AC
:1052300008F042C0F0E0EE5BFE4C32C780E090E048
:10524000D6CE8091F100F701808381E0C81AD108A1
:1052500091F28FEFE81AF80A8091E80085FDF1CF0E
:105260008091E8008B778093E8000E942D0B8115D8
:1052700099F3C1CFE43148F4E11549F0E150E3314D
:1052800030F4F0E0E05BFE4C0BC7EE3F79F28FEFBD
:10529000898312C01A8289E08B830EC08A81823092
:1052A00079F08330A9F0813091F70E941A0AFED676
:1052B0006B837C838D839E83C1010E94970799CD68
:1052C00088E290E03AD71B821C821D828E83F4CF45
:1052D0008091120290911302892B71F38AE0EDE321
:1052E000F2E0DE01139601900D928A95E1F7E4CF8A
:1052F0008A81823061F66B817C818D819E81D6D6D8
:1053000088E290E036D7D8CF4C816B818A810E94A9
:1053100054159827892798278D839E83CDCF2D817B
:105320003E813227232732274C816B818A810E945C
:10533000AF0CC2CF0E943D16BFCF8A81893009F0E1
:10534000BBCF8B8127E0829FC00111246FEF70E0FB
:105350005ED6862F0E947F07AFCF8A81893029F0E1
:105360008A3009F0A9CF1B82A7CF8091930286953E
:10537000869586952FEF829FC001112467E070E02B
:1053800046D66B8399CF83E992E00E94930C94CF29
:1053900080E28A8391CF1A8287E67ECF8C818D311D
:1053A00008F08ACF8A809B80982489249824A12C95
:1053B000B12C61017101E80EF11CCE14DF0409F477
:1053C0007BCF87E688169104A104B10478F4C40168
:1053D00087569C4FB2D6F60184838FEFC81AD80A3D
:1053E0008FEF881A980AA80AB80AE7CF80E0F3CFAF
:1053F0008091120290911302892B09F45DCF0C81E8
:105400000D3108F059CF8A809B80982489249824F4
:10541000A12CB12C71012501320140165104610407
:10542000710408F049CF87E688169104A104B104FD
:1054300030F4F7016481C40187569C4F9AD68FEFF0
:10544000481A580A680A780A8FEF881A980AA80A30
:10545000B80A8FEFE81AF80AE0CF13DB2DCF86E009
:1054600098CF0C810D3108F027CF8A809B8098243B
:1054700089249824A12CB12C250132017E0185E0DC
:10548000E80EF11C401651046104710408F014CFB9
:1054900080ED881682E09806A104B10488F4C40166
:1054A00089964BD6F70181937F018FEF481A580AEE
:1054B000680A780A8FEF881A980AA80AB80AE2CF11
:1054C00080E0F0CF0C81C02ED12C0D3108F0F4CE4D
:1054D0008A819B819827892798274C01A12CB12C80
:1054E000803D22E0920708F0E7CEB50140ED52E0A2
:1054F000481959096A097B09401751056105710569
:1055000008F4DACE2091120230911302232BE1F538
:105510009C01275D3F4F2FA738AB80FB662460F8C6
:10552000712C80FF0AC0889608D62D81382FC901BA
:1055300081159C4711F48FEF8D83C401D501800F35
:10554000911DA11DB11D80FF18C0260181E0481AE0
:1055500051087E0185E0E80EF11CE40CF51C8FA5D6
:1055600098A98C0D9D1DE9D5F7012081922F8115F9
:105570009C4711F48FEF80836201F101E60DF71D66
:105580002FEF6C147D0428F07101612C712C230124
:1055900026C044818581942F81159C4711F4248372
:1055A000258382E0680E711C3296EBCF80ED881661
:1055B00082E09806A104B10428F4F7016481C401D3
:1055C0008996D7D58FEF481A580A680A780A8FEF5C
:1055D000881A980AA80AB80A8FEFE81AF80A40163B
:1055E00051046104710410F367CE8091120290910E
:1055F0001302892B09F460CEC1010E9497078FEF37
:1056000091EE24E0815090402040E1F700C000007E
:10561000C6CB88E0E2E3F1E0DE01919601900D92C5
:105620008A95E1F7FE0132968FE111928A95E9F7AA
:1056300086E0898388E0FE01B196DE01159653CE9F
:1056400088E4898381E08A831B821C8235CE8B812A
:105650009C81A92FAA0FAA0BBA2F25E0880F991FAA
:10566000AA1FBB1F2A95D1F7803E2FEF9207A207F2
:10567000B20708F021CE883421E09207A105B105D8
:1056800008F01ACEAC01BD01405E5F4F6F4F7F4FF7
:10569000493421E052076105710510F048E451E0FA
:1056A000481B590BBC0164537A4FC10110D504CE7D
:1056B0004AE150E06FEF70E0CE01079627D5809168
:1056C00012028983EA821B821C821D8281E0FECD48
:1056D00081E080935A0210925B0282E38093100271
:1056E000109211020E940B0980930E0290930F02F8
:1056F000E3CDE114F104C9F100913D02C0900E0226
:10570000D0900F020E940B098C199D0985369105D6
:1057100098F101FB882780F98BA71CA6802F817048
:105720008DA71EA68BA59CA52DA53EA58223932300
:10573000892B11F10E940B0980930E0290930F02A6
:105740008091100290911102019780931002909322
:105750001102892B51F410925A0210925B0281E0DF
:105760008093120210921302E12C8091120289831D
:10577000EA828091100290CD82E380931002109211
:105780001102F3CF109212021092130295CD40E253
:1057900050E06FEF70E0C101B9D48ECD8B818230C3
:1057A00009F44FC070F4811135C0FE0132968EE1CC
:1057B00011928A95E9F788E089838B8383E088A337
:1057C0007BCD853009F472C0863009F075CD0C812F
:1057D0008AE0FE013596DE01919601900D928A9540
:1057E000E1F78BA19CA10E94A5078BA39CA38FEF3F
:1057F000083060F48AE0089FB0011124675B7C4F99
:105800004AE050E0CE018196D2D480E089830E94A4
:10581000B21652CD8C810AE07E0191E2E90EF11CB4
:10582000F701902F11929A95E9F7B7010E94151789
:105830008983F701DE01129601900D920A95E1F736
:105840003BCD0C818AE0FE013596DE0191960190F8
:105850000D928A95E1F789A19AA10E94A50789A3D3
:105860009AA38BA19CA10E94A5078BA39CA38DA1A9
:105870009EA10E94A5078DA39EA38FA198A50E941B
:10588000A5078FA398A78FEF083060F48AE0089FE0
:10589000B001112467507D4F4AE050E0CE0181965F
:1058A00086D480E089830E94B20706CD6C81CE0148
:1058B0008196FC012AE011922A95E9F7683088F474
:1058C0002AE0269FB0011124675B7C4F4AE050E03C
:1058D00024D480E089838AE0FE01B196DE0112962D
:1058E00002CD8FEFF7CF2B30310508F00CCC39CC3F
:1058F0002B30310508F0C2CBEFCB8091F50181153B
:1059000009F47BCA80E189BD82E189BD09B400FE4A
:10591000FDCF8091D8008F7D8093D8008091E000EA
:1059200082608093E0008091E00081FDFCCF0E94C6
:10593000400D63CA1F921FB61F9211248F939F932D
:10594000AF93BF938091F401811113C08091E10165
:105950009091E201A091E301B091E4014196A11D73
:10596000B11D8093E1019093E201A093E301B09314
:10597000E401BF91AF919F918F911F901FBE1F9027
:10598000189578941F921FB61F9211248F939F939E
:10599000AF93BF938091E1019091E201A091E30167
:1059A000B091E4010196A11DB11D8093E101909396
:1059B000E201A093E301B093E401BF91AF919F9105
:1059C0008F911F901FBE1F9018951F920F920FB6B8
:1059D0000F9211242F933F934F935F936F937F9375
:1059E0008F939F93AF93BF93EF93FF938091E100C9
:1059F00082FF09C08091E20082FF05C08091E10032
:105A00008B7F8093E1008091DA0080FF24C0809139
:105A1000D80080FF20C08091DA008E7F8093DA006A
:105A20008091D90080FFA9C080E189BD82E189BD54
:105A300009B400FEFDCF81E0809314028091D00173
:105A4000811109C00E94AD0B0E945E0B8091E200A3
:105A500084608093E2008091E10080FF1AC0809111
:105A6000E20080FF16C08091E2008E7F8093E2000A
:105A70008091E20080618093E2008091D800806292
:105A80008093D80019BC85E08093140283E0809352
:105A900003018091E10084FF2FC08091E20084FF28
:105AA0002BC080E189BD82E189BD09B400FEFDCF34
:105AB0008091D8008F7D8093D8008091E1008F7E07
:105AC0008093E1008091E2008F7E8093E2008091DC
:105AD000E20081608093E2008091CF01811509F49A
:105AE00052C084E08093140280911402843009F043
:105AF00052C082E0809303018091E10083FF2CC0BB
:105B00008091E20083FF28C08091E100877F80932D
:105B1000E10082E0809314021092CF018091E100B5
:105B20008E7F8093E1008091E2008E7F8093E2007F
:105B30008091E20080618093E20042E060E080E0DA
:105B40000E94DE0A8091F00088608093F00081E07E
:105B50008093030180930201FF91EF91BF91AF9178
:105B60009F918F917F916F915F914F913F912F9175
:105B70000F900FBE0F901F90189519BC1092140231
:105B80001092D00168CF8091E30087FF02C083E0CC
:105B9000A9CF81E0A7CF81E0ADCF1F920F920FB6C2
:105BA0000F9211241F932F933F934F935F936F9303
:105BB0007F938F939F93AF93BF93CF93DF93EF9395
:105BC000FF93E9EEF0E080811091EC008F7010FB04
:105BD000112717F9182B1082C0EFD0E08881877F3A
:105BE000888378940E94730DE9EEF0E0108288813A
:105BF000886088831F701083FF91EF91DF91CF91B0
:105C0000BF91AF919F918F917F916F915F914F91D4
:105C10003F912F911F910F900FBE0F901F901895DD
:105C20008EE1489B02C08150E1F7489BFECF08956A
:105C3000589880E28A95F1F7589A0895FC018BE014
:105C40008A95F1F798E020E080E031E040E14A9564
:105C5000F1F7880F489B02C08160232742E04A95F4
:105C6000F1F7000040E14A95F1F7915079F790E1A2
:105C70009A95F1F799B132E03A95F1F7000030E1E9
:105C80003A95F1F7917092272081920F90830895B1
:105C9000A1E0B0E0EDE4FEE271C119828C017C016B
:105CA000E60EF11CBDDFCE010196C8DFF80181933D
:105CB0008F01EE15FF05B1F781E09981911180E028
:105CC0002196E6E077C1509A589A08955098589ACC
:105CD000E89AE9E6F0E080818C7F80830895615046
:105CE000770B91E001C0990F6A95EAF7692F90E070
:105CF00021E0611108C0911591F0589A80E28A95CF
:105D0000F1F758980895362F382339F0589A92278A
:105D100030E23A95F1F76695ECCF5898F9CF58985C
:105D2000EDCFFF920F931F93CF93DF93EC018C0184
:105D3000060F111D8991F82E7BDF68E08F2DCFDFD4
:105D4000C017D107B9F7CDB7DEB7E5E034C11F9270
:105D50000F920FB60F9211240F931F932F933F931F
:105D60004F935F936F937F938F939F93AF93BF9363
:105D7000EF93FF93CF93DF930F92CDB7DEB71982E6
:105D80004FDFCE0101965ADF082F0695069506953E
:105D9000282F22952570902F9570920F292F237010
:105DA00096959695920F982797708981892B09F07F
:105DB00055C0053008F052C080E18A95F1F7589A35
:105DC000509A82E08A95F1F700C0589888E0089FC1
:105DD00080011124D801AF5EBE4F1696ED91FD9162
:105DE0001897309791F060914A0170914B01149689
:105DF0002D913D91260F371F15978D919D91680F1D
:105E0000791F4C9113978C910995F801EF5EFE4F25
:105E10006381611549F020914A0130914B018481E1
:105E20009581820F931F7DDF03DF80E18A95F1F773
:105E300058985098589A80E18A95F1F7F801EF5EEA
:105E4000FE4F6081611549F020914A0130914B016C
:105E500081819281820F931F1BDFE2DE0F90DF9121
:105E6000CF91FF91EF91BF91AF919F918F917F91D2
:105E70006F915F914F913F912F911F910F910F90D3
:105E80000FBE0F901F9018950F931F93CF93DF9322
:105E9000EC0105970CF05EC0F894509A589885E094
:105EA0008A95F1F700009C2F969595708C2F857040
:105EB000980F892F837096959695292F93E0CC0F94
:105EC000DD1F9A95E1F7280F822F8C2B082FB0DE6B
:105ED00000C068E0802F03DF80E18A95F1F75098D9
:105EE000589A489B30C087E090E048992EC0FE0148
:105EF000EF5EFE4F6381611559F020914A013091A8
:105F00004B0184819581820F931FC2DE8115F9F0C8
:105F100087DE80E28A95F1F75898509A80E18A9559
:105F2000F1F7CF5EDE4F6881611549F020914A019B
:105F300030914B0189819A81820F931FF2DE78DEC6
:105F4000789481E008C000C0CCCF019749F4509A02
:105F5000589A789480E0DF91CF911F910F91089526
:105F600000C0C3CF2F923F924F925F926F927F9269
:105F70008F929F92AF92BF92CF92DF92EF92FF9259
:105F80000F931F93CF93DF93CDB7DEB7CA1BDB0B05
:105F90000FB6F894DEBF0FBECDBF09942A883988AA
:105FA00048885F846E847D848C849B84AA84B984B1
:105FB000C884DF80EE80FD800C811B81AA81B981BD
:105FC000CE0FD11D0FB6F894DEBF0FBECDBFED01D1
:105FD0000895A29FB001B39FC001A39F700D811DC2
:105FE0001124911DB29F700D811D1124911D0895E2
:105FF000DB018F939F9361D0BF91AF91A29F800DE2
:10600000911DA39F900DB29F900D11240895AA1B7E
:10601000BB1B51E107C0AA1FBB1FA617B70710F093
:10602000A61BB70B881F991F5A95A9F780959095C5
:10603000BC01CD01089597FB072E16F4009406D0FD
:1060400077FD08D0E4DF07FC05D03EF490958195FC
:106050009F4F0895709561957F4F0895A1E21A2E84
:10606000AA1BBB1BFD010DC0AA1FBB1FEE1FFF1FFC
:10607000A217B307E407F50720F0A21BB30BE40B4C
:10608000F50B661F771F881F991F1A9469F7609593
:106090007095809590959B01AC01BD01CF0108954D
:1060A000EE0FFF1F0590F491E02D099469279627C4
:1060B000692778278727782708958BDFA59F900D7C
:1060C000B49F900DA49F800D911D11240895FB0194
:1060D000DC0102C005900D9241505040D8F7089560
:1060E000FB01DC0104C08D910190801921F4415025
:1060F0005040C8F7881B990B0895FB01DC0102C0D2
:1061000001900D9241505040D8F70895DC0101C034
:106110006D9341505040E0F70895DC01CB01FC0144
:10612000F999FECF06C0F2BDE1BDF89A319600B4F0
:106130000D9241505040B8F70895F999FECF92BDA5
:1061400081BDF89A992780B50895A8E1B0E042E0B2
:1061500050E0E5CFDC01A40FB51F4150504040F0A6
:10616000CB01840F951F2E9105D041505040D8F798
:106170000895262FF999FECF92BD81BDF89A019717
:1061800000B4021639F01FBA20BD0FB6F894FA9A7F
:10619000F99A0FBE08950396272FECDFEADF252F2B
:1061A000E9DF242FE7CF0196272FE4DFE2CFDC01E0
:1061B000CB0102C02D9105D041505040D8F7089531
:1061C000262FF999FECF1FBA92BD81BD20BD0FB613
:1061D000F894FA9AF99A0FBE01960895F894FFCFB1
:1061E0006F09740976097B098B098B098B098B0967
:1061F0008B098B098B098B097D0981098409890920
:1062000098099E09A209510E770E7D0E770E7D0E1C
:10621000CB0EED0E7D0EF10FFE0F991D011EA11D7F
:106220006B1D6F1DA51D731DA91DB51D7F1DFA1DBD
:10623000831DB91D871DBD1DE21D8B1DC11DE91DDF
:10624000911DC71DCF1D771DAD1D7B1DB11D951D5A
:10625000CB1DD91DF21DF81D651D9D1D081E371D86
:106260003D1D2A1D311D431D491D4F1D421F421F4B
:10627000771F771F22203D20981F981F4220BC20A7
:10628000CD20CD20092B202B272B5C295C29582BD6
:10629000682B792BC22BC72B5C295C295C29CE2B60
:1062A0004A294E29782984298F299A299D29AD299F
:1062B000C3294729F52AC829CB29CE29F8292D2A0F
:0662C0002F2A312A622A98
:1062C60000000100010809640C800A770C7C0C5C54
:1062D6000C000000010000000000000005010000A5
:1062E600000406000000000000010A000000000093
:1062F6000001BBBBAD3D7081F6410044227B4901E4
:106306002701AC009F01B801D8011D02F0F597F6F0
:10631600F7F1F437929394E200E900EA00B500B68B
:1063260000B700CD008301CC008A019201940121BF
:1063360002230224022502260227022A02B300B4FF
:10634600006F0070009F01CB019F02A002E200E9EE
:1063560000EA00B500B600B700CD008301CC008A84
:10636600019201940121022302240225022602271A
:10637600022A02B300B4006F0070009F01CB019F98
:0463860002A002006F
:00000001FF
